:100000000C942A000C943C000C943C000C943C0092
:100010000C943C000C943C000C943C000C943C0070
:100020000C943C000C943C000C943C000C943C0060
:100030000C943C000C943C000C943C000C943C0050
:100040000C943C000C943C000C943C000C943C0040
:100050000C943C0011241FBECFE5D8E0DEBFCDBF1D
:1000600010E0A0E6B0E001C01D92AF38B107E1F7A3
:100070000E9486000C942F010C940000C99B02C0C2
:10008000D99801C0D99A8CB59DB5909361008093A1
:1000900060000895C89B02C0D89801C0D89A8CB55A
:1000A0009DB59093690080936800089580918E00BB
:1000B0008F5F80938E0080918E00893010F01092B7
:1000C0008E00E0918E00F0E0EE0FFF1FEE0FFF1F9D
:1000D000E659FF4F80819181909363008093620085
:1000E000E0918E00F0E0EE0FFF1FEE0FFF1FE659CC
:1000F000FF4F8281938190936700809366008CB557
:100100009DB59093650080936400089544EC50E0A1
:1001100050936B0040936A008AE698E190936D00DB
:1001200080936C0020E137E230936F0020936E00E3
:1001300030937100209370008EE490E090937300F0
:100140008093720084EA97E0909375008093740026
:1001500030937700209376003093790020937800D5
:1001600088E290E090937B0080937A0086E891E0AB
:1001700090937D0080937C0030937F0020937E00DD
:10018000309381002093800088E090E0909383007A
:1001900080938200509385004093840030938700C1
:1001A00020938600309389002093880030938B0041
:1001B00020938A0030938D0020938C0080918A00D8
:1001C00090918B00909363008093620080918C00EB
:1001D00090918D00909367008093660083E08EBDC0
:1001E00087E080938E0080918200909183009093AD
:1001F00063008093620080918400909185009093C9
:10020000670080936600309367002093660088E85B
:1002100093E19093630080936200809162009091DB
:10022000630080519742C9F38CB59DB52091600061
:10023000309161004091620050916300821B930BEA
:100240008417950750F3C99B02C0D99801C0D99A69
:100250008CB59DB59093610080936000DECFF894DB
:02026000FFCFCE
:00000001FF
